:0200000480007A
:100000006F008004732F2034930F80006308FF0378
:10001000930F90006304FF03930FB0006300FF038E
:10002000130F000063040F0067000F00732F2034CC
:1000300063540F006F00400093E19153171F0000BD
:1000400023223FFC6FF09FFF93000000130100008C
:10005000930100001302000093020000130300004C
:100060009303000013040000930400001305000034
:10007000930500001306000093060000130700001C
:100080009307000013080000930800001309000004
:1000900093090000130A0000930A0000130B0000EC
:1000A000930B0000130C0000930C0000130D0000D4
:1000B000930D0000130E0000930E0000130F0000BC
:1000C000930F0000732540F16310050097020000B4
:1000D000938202017390523073500018970200000F
:1000E00093824202739052309B021000939252030B
:1000F0009382F2FF7390023B9302F0017390023AF5
:100100007350403097020000938242017390523046
:10011000735020307350303093010000970200007C
:10012000938282EE73905230130510001315F5017F
:10013000635C05000F00F00F930110009308D005D9
:10014000130500007300000093020000638A0200A0
:1001500073905210B7B200009B82921073902230BD
:100160007350003097020000938242017390123462
:10017000732540F1730020309B00F0FF93907002D4
:1001800013D700409B03F0FF939373029301200069
:100190006314772AB700008013D71040B70300C05C
:1001A00093013000631A7728B700008013D770409E
:1001B000B70300FF9301400063107728B700008069
:1001C00013D7E040B703FEFF930150006316772674
:1001D000B70000809B80100013D7F0419303F0FF1D
:1001E00093016000631A7724B70000809B80F0FFC2
:1001F00013D70040B70300809B83F3FF9301700087
:10020000631C7722B70000809B80F0FF13D710405B
:10021000B70300409B83F3FF93018000631E7720A8
:10022000B70000809B80F0FF13D77040B703000138
:100230009B83F3FF9301900063107720B700008049
:100240009B80F0FF13D7E040B70302009B83F3FFCE
:100250009301A0006312771EB70000809B80F0FF1F
:1002600013D7F041930300009301B0006316771C8D
:10027000B78081819B80101813D70040B78381819C
:100280009B8313189301C0006318771AB78081818C
:100290009B80101813D71040B7C3C0C09B83030CBA
:1002A0009301D000631A7718B78081819B80101862
:1002B00013D77040B70303FF9B8333309301E000F3
:1002C000631C7716B78081819B80101813D7E0409C
:1002D000B703FEFF9B8363609301F000631E7714F6
:1002E000B78081819B80101813D7F0419303F0FFF2
:1002F0009301000163127714B700008093D070401F
:10030000B70300FF930110016398701213020000FD
:10031000B700008013D770401303070013021200C8
:1003200093022000E31652FEB70300FF9301200161
:100330006314731013020000B700008013D7E0406D
:1003400013000000130307001302120093022000A1
:10035000E31452FEB703FEFF93013001631E730CDA
:1003600013020000B70000809B80100013D7F041FB
:100370001300000013000000130307001302120013
:1003800093022000E31052FE9303F0FF930140011B
:100390006314730A13020000B700008013D7704083
:1003A0001302120093022000E31852FEB70300FF6D
:1003B000930150016312770813020000B700008018
:1003C0001300000013D7E040130212009302200034
:1003D000E31652FEB703FEFF93016001631E77042C
:1003E00013020000B70000809B8010001300000083
:1003F0001300000013D7F0411302120093022000F3
:10040000E31252FE9303F0FF93017001631677022B
:10041000935040409303000093018001639E70005D
:100420009300100213D0A0409303000093019001A9
:1004300063147000631030020F00F00F638001003E
:100440009391110093E111009308D00513850100E9
:10045000730000000F00F00F930110009308D00507
:100460001305000073000000731000C000000000BE
:0C04700000000000000000000000000080
:1010000000000000000000000000000000000000E0
:1010100000000000000000000000000000000000D0
:1010200000000000000000000000000000000000C0
:1010300000000000000000000000000000000000B0
:081040000000000000000000A8
:040000058000000077
:00000001FF
